:030000000219FDE5
:03000B000200A848
:03002B0002015D72
:03005B000202DCC2
:030073000202C2C4
:1000800002030406080C10182030406080040608A3
:100090000C10182030406080A0C000070F1F3F05E3
:1000A000050D050205030302C2AFC0D0C0E0206207
:1000B00017E5256002E473E525F4F58A758B00D217
:1000C00062D0E0D0D0D2AF3285268AC262E526F473
:1000D000602F758B00D0E0D0D0C294C292C290D273
:1000E000AF32C294C292C290206E0C206609740591
:1000F000D5E0FDE57E4290758B00D0E0D0D0D2AF48
:1001000032758A00C28DD26201F701B730680520CE
:100110006602D29401B7306805206602D29201B718
:10012000306805206602D29001B7C29530680A2077
:1001300066077428D5E0FDD29401B7C29330680AEF
:100140002066077428D5E0FDD29201B7C2913068CD
:100150000A2066077428D5E0FDD29001B7C2AFC26D
:10016000AD53E6EFC0D0C0E0D2D3D2AFC2CEE52AC5
:100170006007207449152A21BE7800790020742E6A
:10018000E580307E01F430E40278FF53DACF207E40
:100190000343DA20307E0343DA10C2D8C271E5800F
:1001A000307E01F430E40279FFC3E89970CB30610E
:1001B00003752A18207403752A18885FD27020747A
:1001C0000DE52B6004152B21CE43DA01C2D8207037
:1001D000024130A85F206102C270207431C3E894EC
:1001E000F0400374F0F8E8C4540F28F87984B7039A
:1001F00002410EC313C3138721200802C313200A30
:1002000006C3C898F8410E28F8500374FFF8C3E8F5
:1002100095685003E568F88822E52D54066011E5DD
:1002200033C313C31324062522F52250037522FF7E
:10023000852224A824C3E52495644002A864882567
:10024000E56970024174C3E8AA699A5003E8FAE4C8
:10025000F9EAC333FBE56BF45B29400D256AF8E549
:100260006A6002156A400B41740AC3E56A9A50023B
:10027000056A78FF8826C3E52594404002D26420B1
:10028000CF0AD0E0D0D043E610D2AD32C2CF053A8B
:100290007801E52A6005307402152AC3E55F9401F0
:1002A000400575620041B8756300756C00E5622415
:1002B00001F56250037562FFD0E0D0D043E610D262
:1002C000AD32C2AFC0D053E67FC260759100855693
:1002D00094855795759104D0D0D2AF32C2AF53E612
:1002E000EFC2ADC0D0C0E0C0F0D2D3D2AFA8FBA95E
:1002F000FCC2D8307102614353DACF207E0343DA67
:1003000010307E0343DA20D271E580307E01F42084
:10031000E402611A88278928A17053DACF207E036E
:1003200043DA20307E0343DA10C2D8C2713074023F
:10033000A15C7800E580307E01F430E402A15C88A5
:100340005FA14453DACF207E0343DA20307E03439B
:10035000DA10C271206102811C53DACF207E034380
:10036000DA10307E0343DA20C2D8D271885A895B12
:10037000C3E89558F8E99559F97B007E087A00C3DF
:10038000E8948CE994005005755E00810E88217810
:10039000A2E6A8216055C3E894C8E994005008E497
:1003A000D2E4FB7A0A61E9C3E89468E99401500851
:1003B000E4D2E3FB7A0F61E9C3E894D0E9940250F8
:1003C00008E4D2E2FB7A1E61E9C3E894A0E994054F
:1003D0005008E4D2E1FB7A3C61E9C3E89498E994DF
:1003E000085008E4D2E0FB7A787E00C3E8955CFC14
:1003F000E9955DFD30E70AECF42401FCEDF43400EE
:10040000FD755E00C3EC9AED9E5003755E01885C3D
:10041000895D855A58855B597802A144C3E89527C0
:10042000F8E99528F9307C02A128307B02A1283018
:100430007A02A121207502813FE9FDE8FC815EE995
:10044000C313F9E813F8307902A121E9C313F9E8DD
:1004500013F8307802A121E9C313FDE813FC2061F1
:100460002CC3EC941CED940240028175ED701EC308
:0E047000EC94C850180529E52970021529C31F
:10047E00E529940A5002A15C755F00D270A15CE57B
:10048E0029600215297888E6F97400207F0878968D
:10049E00B90302789EE624FAFEE43400FFC3EC9E14
:1004AE00FCED9FFD9208B90310A2085007207609B3
:1004BE00D27681C7307602C276A2085016B9030DE5
:1004CE00ECF42401FCEDF43400FD0204E178007933
:1004DE0000A128B90315EC33FCED33FDC3EC940AEF
:1004EE00FCED9400FD50047C007D00C3EC94FFED08
:1004FE009400400678FF7900A128EC8575F0A4C51C
:10050E00F0A2F733F87900400302054478FF790032
:10051E00020544E9C313F9E813F8307C0EE96002D2
:10052E0078FFC3E81338F8E43400F9C3E894FFE920
:10053E009400400278FF885FD270206102A15C7443
:10054E001FF4552F4BF52FC274EB7002D274752A1F
:10055E0018307403752A0A306102A1702074035397
:10056E00DAFE207403752B06D0F0D0E0D0D0D2ADD9
:10057E0043E6103279010205A079030205A0790A3B
:10058E000205A0791E0205A079640205A079C802B1
:10059E0005A07817E4D5E0FDD8FAD9F6227A147BB7
:1005AE00780205C77A107B8C0205C77A0D7BB402E0
:1005BE0005C77A0B7BC80205C77902B27DE4C293E8
:1005CE00D5E0FDD292D5E0FDC292D5E0FDD293D515
:1005DE00E0FDD294E576D5E0FDC2947496D5E0FDAB
:1005EE00D9D9EAF8D5E0FDD8FBDBCEC29322C37C85
:1005FE00007D0075F00005F0EA33FAEB33FB50F6A0
:10060E00EB13FBEA13FAC3E9FFE8FEE89AF8E99B5D
:10061E00F95004EFF9EEF8B3EC33FCED33FDD5F001
:10062E00DFEDF9ECF822E889F08A20D2D4F8A9F0AF
:10063E007B0030F70B7BFFF42401F8E9F43400F96A
:10064E00E88520F0A4ADF0F8E98520F0A4AFF0FE27
:10065E00ED2EF974003FFA7C04C3EA13FAE913F99C
:10066E00E813F8DCF48BF030F70AE8F42401F8E92B
:10067E00F43400F9E889F0C2D4F8A9F02222C3E5D7
:10068E004113F9E54013F8C3E54598F8E54699F9A5
:10069E00500CC3E89480E994FF40160206C3C3E8E9
:1006AE00947FE9940050030206C3787F7900020616
:1006BE00C3788079FF884A894B22E54A2547F8E5B9
:1006CE004B3548F9854B20E4300701F43549FA30B3
:1006DE00E709C3EA94F04015020701C3EA940F50EC
:1006EE000302070178FF79FF7A0F0207017800797C
:1006FE00007AF0C3E5249564500AC3740195245022
:10070E000B02071FE54B20E70E02071FE54B30E7F4
:10071E0006884789488A492278A4E6FAC3E54A330F
:10072E00F8E54B33F9D134E930E70BC3E89480E9AF
:10073E0094FF4013E159C3E8947FE994005002E11D
:10074E0059787F7900E159788079FFE820E715C361
:10075E00E52398F84009C3E8940140030207807826
:10076E0001020780E8F424012523F84003020780E4
:10077E0078FF884C2278A5E6FAA848A949D134E931
:10078E0030E70CC3E89401E994FF40160207B4C3A6
:10079E00E894FFE9940050030207B478FF79000251
:1007AE0007B4780179FFE920E715C3E54C98F840C6
:1007BE0009C3E8940140030207DB78010207DBE876
:1007CE00F42401254CF840030207DB78FF8824222D
:1007DE0078FFC26420693D206A12D264C3E5419459
:1007EE000A4009C3E52594405002C26479A1E7602E
:1007FE0023E541601F74FF8541F0848539F0306A2E
:10080E000375F005A4F8C5F0600278FFC3E895679C
:10081E005002A867886622C3E5409440E5419401E2
:10082E00E5665003140136046002F5662202083EA6
:10083E002275E890227883E6FFE5E820ECF7A8BD64
:10084E00A9BE0573C3E57394084052757300E9FAA7
:10085E0079A0E76044EA7007E574601B020879C36B
:0F086E00E895746010E5745006600C140208855C
:10087D000460F9020885E574F574C3946D401B7529
:10088D0064C0C394044013756480C39404400B7515
:10089D006440C39404400375640075BB0E22E56487
:1008AD00F460020564E573B4070375BB102274325E
:1008BD0079A687F0A4C5F0A2F733F8C3E895644094
:1008CD0002A8648822882488258826886722754096
:1008DD00007541F022C2AF75C820A8CCA9CDAA3AA7
:1008ED0030CF010A75C824D2AFAB3BAC3C883B89F5
:1008FD003CC3E89BF8E99C206908F930670221F7B1
:10090D002154AD3D8A3DF9EA9DFA600478FF79FFE7
:10091D00AE3EAF3F8B3E8C3FC3EC9FFCC3E99CF5D5
:10092D0042A83BA93CC3E89EF8E99FF9C3E54113F2
:10093D00FBE54013FAE82AF540E93BF54150067511
:10094D0040FF7541FF219EAA40AB41AC40AD417EB9
:10095D00047F02C3EB940440021E1FC3EB940840B6
:10096D00021E1FC3ED13FDEC13FCDEF7C3EA9CFA68
:10097D00EB9DFBEF6009C3E913F9E813F8DFF7EA24
:10098D0028FAEB39FB8A408B4150067BFF8B408B5D
:10099D0041C3EB94025002D2673069047F0321C931
:1009AD007892E6FFC3E537948240110FC3E5379483
:1009BD00A040010FC3EF940640027F057E07E5417D
:1009CD00C4540FF9E541C454F0F8E540C4540F2860
:1009DD00F8C3E89EFAE99400FB4009C3EA9402EBE0
:1009ED00940050047A02E4FB4143AA40AB41EBC4AE
:1009FD00FEEAC4540F4EFCC3EA9CFAEB9400FBC311
:100A0D00E813C313F8EA28FAEB3400FB8A408B4154
:100A1D00C3EB94024002C2677807EBC4FE7B00EA89
:100A2D00C4540F4EFAC3EA98FA4005C3940250021B
:100A3D007A027892E6FF3060024143855256855323
:100A4D0057D26043E680C3E49AF8E49BF93067021D
:100A5D0041DDE8FAE9FBD3E913FDE813FC8852897F
:100A6D0053C3EF94036038EF20E00DE82CF8E93D17
:100A7D00F9ECFAEDFB020A98E828F8E939F9C3E830
:100A8D002402F8E93400F97AFE7BFFC3EF940340AA
:100A9D000E8A548B55884E894F8C508D516111881B
:100AAD005489558A4E8B4F8C508D51306920C3E53A
:100ABD003394034019E542A2E713F8E555F42401F8
:100ACD0038400B20E7087554FFF42401F5556111EA
:100ADD00E8FAD3E813FC8852C3EF94036020EF20AB
:100AED00E007E82CF8ECFA41FDE8282402F87AFE3C
:100AFD00C3EF940340088A54884E8C50611188547A
:100B0D008A4E8C50E56BC3335002646BF56B3060CD
:100B1D0002611B753402D26043E680E52D540660F8
:100B2D0026A840A941C3E913F9E813F8C2AF53E66B
:100B3D007F759100C3E498F594E499F5957591044A
:100B4D00D26043E680D2AF22D26575440075200095
:100B5D00306B03752040020B74D26575440075200F
:100B6D0040306B03752000D2AF7801206722E52D50
:100B7D0054066002C265C3E54194054013780294A2
:100B8D000540087803940540027806306902780A1A
:100B9D00206019E544601530690AC3E533940340BC
:100BAD0003D53406D2AFD26C81467123D2AF00008B
:100BBD00C2AF206726E541C3FB940F40027B0FEBCC
:100BCD00240530730123306A02742820620123F951
:100BDD003069027982E58BC39940B50544E59BF4F4
:100BED005440B52002813030690A08C3E8940A40A8
:100BFD000108619D2065026174C26553E67F7591A0
:100C0D00003067107594007595FE759104D26043A0
:100C1D00E6806174AE40AF41C3E49EF594E49FF568
:100C2D00958117C3E53394025002617430650261FA
:100C3D0074D8028144619DC26C53E67F7591008525
:100C4D005494855595759104854E56854F57D260B0
:100C5D0043E680D2AFE52D54066008206A020533C5
:0E0C6D00020C80306C0D206B0A20650715818B
:100C7B0015810214F7227800306405306502780183
:100C8B00E53775F007A4F9E5F028F5F0E9A2F013C4
:100C9B00A2F113A2F213F537C3947850037537788A
:100CAB00C3E53795384008D266C294C292C29030E1
:100CBB00600281BA855056855157D26043E6802237
:100CCB00207D11C2AF754302C293D295D2AF759FEF
:100CDB0070020E9AC2AF754302C293D291D2AF7516
:100CEB009F70020E9A307243207D20C2AF75430372
:100CFB0090013B757E08C290C291306204D292A1E2
:100D0B000ED293D2AF759F00020E9AC2AF754303FA
:100D1B0090013B757E08C294C295306204D292A1B9
:100D2B002ED293D2AF759F20020E9A207D17C2AFA1
:100D3B00754303900116C290306202D292D2AF7506
:100D4B009F00020E9AC2AF754303900116C29430F6
:100D5B006202D292D2AF759F20020E9A207D11C2F1
:100D6B00AF754304C295D291D2AF759F20020E9AF4
:100D7B00C2AF754304C291D295D2AF759F00020EDC
:100D8B009A307243207D20C2AF75430590012A75BE
:100D9B007E20C292C293306204D294A1AAD295D281
:100DAB00AF759F70020E9AC2AF75430590014C75DB
:100DBB007E02C292C293306204D290A1CAD291D267
:100DCB00AF759F70020E9A207D17C2AF75430590C9
:100DDB00010CC292306202D294D2AF759F70020E98
:100DEB009AC2AF754305900120C2923062EBD2904C
:100DFB00D2AF759F70020E9A207D11C2AF7543065C
:100E0B00C291D293D2AF759F00020E9AC2AF7543B7
:100E1B0006C295D293D2AF759F20020E9A307242C2
:100E2B00207D20C2AF75430190014C757E02C294A8
:100E3B00C295306204D290C146D291D2AF759F2039
:100E4B00020E9AC2AF75430190012A757E20C290A3
:100E5B00C291306204D294C166D295D2AF759F0015
:100E6B00C19A207D16C2AF754301900120C2943008
:100E7B006202D290D2AF759F20C19AC2AF75430167
:100E8B0090010CC290306202D294D2AF759F00C217
:100E9B00662290010A757E00C294C292C290C295DE
:100EAB00C293C291C26222788076FF0876FF0876E1
:100EBB00FF0876FF087603087604087609087601A2
:100ECB00087601087601788C76010876FF0876FFA4
:100EDB000876FF0876FF0876FF0876030876FF088A
:100EEB0076FF0876FF0876250876D00876FA08761E
:100EFB00FA0876040876FF08760108760008767AF9
:100F0B000876FF087601087601087600087603223A
:100F1B007887E6FFC2727888E6C394036008C27DC7
:100F2B00E630E102D27DC27E7889E630E102D27EE4
:100F3B00C3EF94026008758E01D273020F4E758E4B
:100F4B0000C273227880E6149000809378A4F67820
:100F5B0081E6149000809378A5F67886E6149000CD
:100F6B008D9378A6F6789CE67538FF75390CB4022C
:100F7B00067538A075390AB40306753882753905BC
:100F8B0078A3E61490009A93F569D19D2222789666
:100F9B00E6FA7897E6FB7888E6B40305C3EB940E84
:100FAB00FB307F047A007BFFC3EB9AFCC394825027
:100FBB00027C827575000575EC8575F0A4C3E5F0B0
:100FCB00947D40F222D27FF1991205917A007B0039
:100FDB007C10120587E55F2AFA74003BFBDCF37C7F
:100FEB0004C3EB13FBEA13FADCF7FEC27FF1992281
:100FFB00E5EF20E6037520000520903FFFE5201468
:10100B006006901DFF1460009304600375EF12538C
:10101B00D9BF7581C043FF8012058275EF0243B2C1
:10102B0003E5B3240420E70DF521E5E320E0068575
:10103B0021B343E301120E9D7580FF75A40075F17A
:10104B00DC75D4EF7590C075A53F75F23F75D5C0B3
:10105B0075A60175E241E4F8F6D8FD756B01120E29
:0D106B00B212153978988676753001C2AF43
:1010780012059B1205AB1205911205B212059112C9
:1010880005B912059112165212059B12059B1205FD
:1010980096C2AF78FA79FA308407D9FBD8F7021CE0
:1010A80000120F1B120F4F120F98120F9978988683
:1010B80076120E9D75885075891275C8247591042D
:1010C80075D84075A82275B80275E690759B80752D
:1010D8009D0075D10E75BC5875BB0E75BA1175E8B3
:1010E80080120582D2AF12083B53DACF207E034329
:1010F800DA20307E0343DA1043DA01C2D8C2711213
:10110800059BD2617B037A0CE55E70077A0CDB03E2
:10111800021099120591207003021099C270E55FC0
:10112800C3940240E1E52F541F856160F561B56005
:10113800D5DAD5C26153DACF207E0343DA20307E78
:101148000343DA10C2D8C27178A2E67008D274E5F7
:101158002F54E0F52FC275752900120596307409D1
:10116800C3E529940A4002D27512058778023074C3
:10117800027800C3E55F9840F0C2AF1205AB1205D4
:10118800AB1205ABD2AF12059B754D007888E6B45B
:1011980003024179120587788CE6C3940150030253
:1011A8001279E530C394015003021279207435C3D3
:1011B800E55F94FF5003021279C2AF1205C0D2AFA7
:1011C800120596C3E55F940150EFC2AF1205AB124A
:1011D800058C1205ABD2AF120596C3E55F94FF40AC
:1011E800E90216D77F05D27F120F99120596C2AF72
:1011F800C27F120F99AE5FC3E55F947FD2AF407B89
:10120800120582C2AF1205C0D2AFDFDA120FD0C307
:10121800EE94057897F612059B12157B12165A7FE5
:101228000AD27F120F99120596C2AFC27F120F9988
:10123800AE5FC3E55F947FD2AF50E4120582C2AFC0
:101248001205AB12058C1205ABD2AFDFD4120FD04A
:10125800EE24057896F612059B12157B1216891254
:101268000596120F99C3E55F94FF500221B4021648
:10127800D7C3E55F954D4003855F4D12059678010C
:101288007988E7B403027805C3E55F9840022194A2
:10129800C2AF1205C01205C01205C0D2AF12059B1D
:1012A800753000E4F531F5320531E531F470390572
:1012B80032789AE67819146012783214600D787DC5
:1012C80014600878FA146003753200C3E532984058
:1012D8001715327531B478998676C2AF1205C0D227
:1012E800AF7898867612059612058CE52A70053037
:1012F8007402019978012074027806C3E55F98406A
:10130800A77888E6C394036003120596E52A70035C
:10131800021099C2AF120E9DE4F522F523F524F5CB
:1013280025F526F56AD2AF7885E6C333F568E4F586
:1013380045F546F547F548F549F573F52CF52DF5CE
:101348003775730875BB1012058212083FE5E8204F
:10135800ECFBA8BDA9BEE97001F8887412084375B2
:10136800730875BB107887E6FE7602120F1B788724
:10137800EEF6C2AF7564FF1208BB8522648522654C
:10138800852266D2AF75220175240175250175265F
:101398000185636C756D017888E6B40307C27D30FA
:1013A8007602D27DD268D269753300120E03120E0E
:1013B800281208DB1208E21208DB1208E21208DB26
:1013C8000213D8C2AF120F1BD2AF75730075BB0ED4
:1013D800120B6612068B120C81120CCB1208E21249
:1013E8000B55306D0312068C2067031207DE306739
:1013F80003120825120C81120CF01208E2120B6677
:10140800306D031206C8120C81120D671208E21221
:101418000B55306D03120726120C81120D8C120821
:10142800E2120B66306D03120783120C81120E0351
:101438001208E212083F120B55120C81120E2812E4
:1014480008431208E2306932206B2F85676485678C
:101458006585636C756D0179187A0CC3E53399401D
:0E1468000CC269D26A8A357564FF021482C311
:10147600E55F940140030213D80214FF306A1B2073
:101486006B18E535147004C26A61CBF535C3E55FA8
:10149600940140030213D80214FF753600C3E562B7
:1014A6007882985054307404E52A604D7888E6B402
:1014B6000317207D0520760781CF30760281CF2065
:1014C6006B07D26B856764811778F0306B0585678B
:1014D600647820C3E54198500261D8306B1BC26B1B
:1014E600C27D307602D27DD26A7535128567646117
:1014F600D80536E55F6002A102753600C2AF120E4E
:101506009D7887E6FE7602120F1B7887EEF6E4F5E5
:1015160022F523F524F525F526F568C268D2AF1223
:101526000582120E9D307409C3E53694054002010A
:101536009941AB901A0D78201215BDE520B45A0CCE
:10154600A31215BDE520B4A50302155B120EB21257
:10155600157B02157A901A0378807B0A1215BDA3B3
:1015660008DBF9901A0F788C7B181215BDA308DBDF
:10157600F9901A2722C2AF1215FC1215D6901A003E
:10158600740E1215C2A374041215C2A37414121594
:10159600C2901A0378807B0A1215C1A308DBF99062
:1015A6001A0F788C7B181215C1A308DBF912160FD7
:1015B6001215ED901A2722E493F622E6438F015383
:1015C6008FFD75EF0275B7A575B7F1F0538FFE2243
:1015D600438F02438F0175EF0275B7A575B7F1907A
:1015E6001A0DF0538FFC22901A0D745AB1C2901A3C
:1015F6000E74A5B1C2227A3079D07820901A40B103
:10160600BDE520F709A3DAF7227A3079D0901A409F
:10161600E7B1C209A3DAF922AB77A878BB01027950
:1016260084BB02027985BB03027986BB04027992E8
:10163600BB05027987BB060279A3BB0702799CBB6F
:1016460008027988BB09027989E8F7227C05120528
:101656009BDCFB22C2AF1205AB1205B21205B91212
:1016660005C012058C1205AB1205B21205B912059A
:10167600C012058C1205AB1205B21205B91205C0CF
:10168600D2AF22C2AF1205C01205B91205B21205B9
:10169600AB12058C1205C01205B91205B21205ABC4
:1016A60012058C1205C01205B91205B21205ABD28D
:1016B600AF22AE77AF78C2AF1205AB1205AB1205FB
:1016C600AB12058CDEF21205C012058CDFF8D2AF24
:1016D60022D15AD152D152757701757801757900A8
:1016E600D1B87C05AD5F12059BC3ED955F70F5C360
:1016F600E55F9401400AC3E55F94FF403202171389
:10170600D11EB17BD15AC2AF75EF12D152DCD505CD
:1017160079C3E5799403500280C6D1520578E577FE
:101726001490009F93F808C3E57898500280AED1D4
:1017360052D1520577C3E577940A5002809C120E67
:0A174600B2B17BC2AF75EF12D152B1
:0319FD00020FFBDB
:101A00000E0414FFFFFFFF0304090101015AA501A1
:101A1000FFFFFFFFFF03FFFFFF25D0FAFA04FF01DE
:081A2000007AFF01010003FF41
:101A40002348694D6F64656C436F6F6C343141237B
:101A500023424C48454C4923463333302320202031
:101A60002020202020202020202020202020202076
:101C0000C2AFC2D353D9BF7581C043B20343FF8073
:101C1000752438752503B1C975EF0275E24043F1AB
:101C20001053A4EF75D400D2847DFA780379E67C52
:101C300010752200752300901DD67B0675249875BB
:101C400025013084028142208408D8FBD9F9DCF7D1
:101C500081B4308408D8FBD9F9DCF781B4B189E4C8
:101C600093A3C39A6004DDC381B4DBDBB17B600264
:101C7000812B7B08E493FAA3B15CDBF87A30B15C8A
:101C8000752200752300B17BEAFCEBFDC3ED94FEE9
:101C9000400EB17B8A278B28ED30E0048A828B834B
:101CA000B17B7AC270D8C3ED94FE601350CEBD00F4
:101CB00025EC60097520007521FF0200008100A855
:101CC00027A9280809D804D90281D3B17FEA89AAB3
:101CD000F281C50D81A0C3ED94035049EDA2E092BD
:101CE000007AC5C3E5829400E583941C50902000DF
:101CF00010438F02438F0175B7A575B7F1F030001F
:101D00001FA827A9280809438F01538FFDD804D99C
:101D100002A12089AAE275B7A575B7F1F0A3A10DBC
:101D2000538FFC817C7AC1BD030CE493A3FAB140CC
:101D3000DCF8B138817C817EAA22AB23B15CEBFA5E
:101D4000EA6222752608C3E52313F523E52213F57D
:101D50002250066323A0632201D526EAB1C9B1C986
:101D600075260AEAF4200102D284300102C284B14D
:101D7000C9C3134002C201D526EB22B17FEAFB2082
:101D80008402A17F308402A184752608AE24AF2589
:101D9000C3EF13FFEE13FEB1CDB1C9C3EA13308414
:101DA000024480FA30E703632201C3E52313F523DD
:101DB000E52213F52250066323A0632201D526D91C
:101DC000E52265236523F52222AE24AF250E0FDE22
:101DD000FEDFFCD20122424C48656C693437316326
:041DE000F3300601D5
:00000001FF
